:020000040000FA
:0400000072303A28F8
:08000800A000030EA100831209
:1000100005191028831601178312B23081002B288E
:1000200083160113831203140B190310A80DA90DD5
:10003000AA0DAB0DAC0DAC16FF302C02031D2B2806
:10004000FA302B02031D2B2831152A08AF0029088E
:10005000AE002808AD008B100B11210E8300A00EFE
:04006000200E090065
:0C007400203084008001840A80300402E7
:10008000031C3C281230B000522183160C30850529
:1000900087018312850187010730990000309A009B
:1000A000103083168E008312603083168F00831207
:1000B0000030831691009F008312C83083168100A0
:1000C000831231309000003083168C008312103080
:1000D0008B00702181018E018F010B118B100B1091
:1000E0008C018B178220311985203421B30B802895
:1000F000031085190314B90DF03039020319DD20FE
:100100007121722864003210080031110130B700EB
:100110008B132030370783169B001C141A08831298
:10012000A4001030370783169B001C141A08831292
:10013000A300A6000230A6060030370783169B00F6
:100140001C141A088312A200A7000130A7068B17FF
:10015000321CB02822090339A200A309A409A50969
:1001600024082F02031DD72823082E02031DC528AB
:1001700022082D02031DD72801303702031DC52890
:100180003D18C5283D143E146A2126082E02031D81
:10019000D72827082D02031DD72801303702031D59
:1001A000D6283D1CD6283D103E146D21D728B70A0D
:1001B000023037020318080088280130B600B30067
:1001C000B400B500B70085018701B1138220B30BDD
:1001D0000329031085190314B90DF03039020319EE
:1001E0002A29B41F8501B41F8701B40B03293708DE
:1001F000B6080319B60003190129FF3085008700EE
:10020000B6039630B400311DE6283111321C0D2999
:100210002D090339AD00AE09AF092F1CE6288E0168
:100220008F010C1CE6280C102E1EE6288B132030A4
:100230003707BB002F08BA003D2110303707BB003D
:100240002E08BA003D2100303707BB002D08BA0048
:100250003D218B1785018701B70AB60102303702AD
:10026000031CE628702108003E1C08003E101030D8
:10027000BB003D08BA003D2108008B133A088316E5
:100280001C159A0083123B0883169B0055309D0075
:10029000AA309D009C1464009C184B291C118312E9
:1002A0008B170800831610309B001C141A08831249
:1002B000BD00FF30D4000230D5000C30D600BA307B
:1002C000D7003730D800DA30D9006F30DA00B830D4
:1002D000DB0008000130BD0008008501870108002F
:1002E000080001303D05031908005C180516DC18EC
:1002F00085165C190514DC1985145C1A8714DC1A40
:1003000007155C1B0714DC1B87165D180716DD1824
:100310008715E6300E02031C97290516851605146D
:1003200085148714071507148716071687158F0875
:10033000031908008F01850187015408DE0024227B
:10034000D4005508DE002422D5005608DE00541CD7
:100350002422D6005708DE00D41C2422D7005808D7
:10036000DE00541D2422D8005908DE00D41D2422AA
:10037000D9005A08DE00541E2422DA005B08DE0091
:10038000D41E2422DB00CA0BCD295408CA00D4187D
:100390005C14D41E5C10D41D5C10CB0BD7295508FF
:1003A000CB00D51ADC14551DDC10551FDC10CC0B0E
:1003B000E1295608CC00561A5C15561F5C11D61D53
:1003C0005C11CD0BEB295708CD00571ADC15D71F50
:1003D000DC11D71DDC11CE0BF5295808CE00D81B37
:1003E0005C16D81F5C12D81C5C12CF0BFF29590871
:1003F000CF00591ADC16591EDC12D91FDC12D00BA3
:10040000092A5A08D000DA195C17DA1D5C135A1E43
:100410005C13D10B132A5B08D1005B1ADC175B1E3F
:10042000DC13DB1FDC13D20B1B2A5608D200D51BB2
:100430005D14D71F5D10D30B232A5708D300D61B9A
:10044000DD14D81FDD100800C001DE080319DE032B
:100450005E184014DE1A40144008C0015E1C4014AF
:0C046000DE1E4014C005C00C5E0C08003D
:084000000F000300050005009C
:02400E00CC33B1
:10420000010078007A007C007E007B0079007F004E
:104210007D007A0078007E007C00FF00FF00FF0038
:104220000000F200F600FA00FE00F200F600FA00CC
:10423000FE00F200F600FA00FE00FF00FF00FF00A3
:10424000010005000500050005000900090009003E
:1042500009000D000D000D000D00FF00FF00FF0024
:10426000FF00FF00FF00FF00FF00FF00FF00FF0056
:10427000FF00FF00FF00FF00FF00FF00FF00FF0046
:10428000FF00FF00FF00FF00FF00FF00FF00FF0036
:10429000FF00FF00FF00FF00FF00FF00FF00FF0026
:1042A000FF00FF00FF00FF00FF00FF00FF00FF0016
:1042B000FF00FF00FF00FF00FF00FF00FF00FF0006
:1042C000FF00FF00FF00FF00FF00FF00FF00FF00F6
:1042D000FF00FF00FF00FF00FF00FF00FF00FF00E6
:1042E000FF00FF00FF00FF00FF00FF00FF00FF00D6
:1042F000FF00FF00FF00FF00FF00FF00FF00DD00E8
:00000001FF
